S06C0000433A5C446F63756D656E747320616E642053657474696E67735C686F6F7665725C4465736B746F705C4543453333312054322046616C6C20323030395F31305C74686572656D696E5C62696E5C5026455F4D756C74696C696E6B5F4379636C6F6E6550726F2E61627332
S1234000000A4B9CCF1000180B01004D180B8000464C40014C4C01180B0100491D0272014D
S12340204D8D014C8280CEFFFF0926FD180B080083180B010084180B8000854F8680FCDCB0
S123404090CD159C1813B34002B745B7642403830001B34000B746B754CE03E81814B76471
S1234060D3445C50180B01004E10EF20FE180B8000854F8680FCDC90CC0147CD159C181348
S1234080B34002B745B7642403830001B34000B746B754CE03E81814B764D3505C50180B78
S10740A001004E0BBE
S105FFEE406D60
S105FFFE4004B9
S9030000FC
